:020000009E2838
:080008008C00030E8D000408BA
:100010008E000108A3000B1D16280B11A40A031D56
:100020001828A50A031D182826212114A1158B01C3
:1000300005091C3903191E28050895000E088400BF
:100040000D0E83008C0E0C0E09000F398207303420
:10005000313432343334343435343634373438345C
:10006000393420342B342D342C342E345F34820731
:1000700050344934433420344334413450342034F0
:100080004D3445345434453452340034463472349B
:10009000203454346F346D3420344D346334473459
:1000A0006134683465346534003441345534543433
:1000B0004F34523441344E34473449344E3447344B
:1000C0002034203420342034203400344F3456344B
:1000D000453452342D34523441344E34473445344F
:1000E000213400344D3441344E34553441344C3491
:1000F00020344D344F3444344534003420342034DB
:10010000203420342034E4346634203420346E34F7
:100110006634203420347034663400345A34453424
:1001200052344F34203441344C344C342034523423
:1001300041344E34473445345334003483161C3034
:10014000850001308600811301138112011281158F
:100150000111811001108312A101A201FF3095004D
:100160008B2300303223B1230E303223E923E923DD
:10017000A523563032230C210821162108211C21E9
:100180000821262108217722D3208B01211C8629D2
:10019000A5232E303223C32805091C390319080072
:1001A00005089500D92805091C390319D92805081F
:1001B000950015091C39031908002210151AEE289C
:1001C00026082A3C031DE6281621002926082D3C76
:1001D000031DEC281C210029262100299519FE2841
:1001E0002608333C031DF6281C2100292608303C34
:1001F000031DFC28162100290C210029772230211B
:1002000005091C39031D0029FF3095002214C3285D
:10021000ED2377223021AA2B221808002A30A600CD
:10022000961416088600051085100800221808008C
:100230002D30A600961011292218080096101608D5
:100240008600051485103030A6000800221808002A
:10025000961016088600051485143330A600080091
:100260002608840023088000840A24088000840A69
:1002700025088000080029082502031942290318CF
:100280005029672928082402031947293F292708EC
:10029000230203194C293F29A301A401A501080049
:1002A00021162708A30203195D2903185D290130CF
:1002B000A40203185D290130A5022808A40203192D
:1002C000642903186429A5032908A5020800270842
:1002D0008F002308A7000F08A30028089000240817
:1002E000A8001008A400290891002508A9001108F9
:1002F000A500502121120F08A7001008A80011081E
:10030000A900AD23FF30BC23ED230800260884009C
:100310000008A700840A0008A800840A0008A900B1
:100320003B212308031999299000FC229003031D07
:10033000952924080319AA2990000630FD220530CA
:100340008F000130FF2202308F000230FF22900325
:10035000031D9D2925080319C32990000630FD229D
:1003600003308F000130FF2205308F000230FF2262
:1003700005308F000330FF2206308F000430FF224B
:100380009003031DAE2926082A3C031DD6295723B6
:10039000532308304C234B23AA233130BC2349225A
:1003A0002508073C0318252A2621242A26082D3C47
:1003B000031DF429572357235723532308304C2375
:1003C0004B23AA233230BC2349222508073C0318BB
:1003D000EB292621242A2508031D252A2408103C60
:1003E000031C252A0C21242A2608303C031D112A2F
:1003F000572357234F23083054234B23AA2333304A
:10040000BC2347222508073C0318082A2621242A52
:100410002508031D252A2408103C031C252A162123
:10042000242A5723572357234F23083054234B2381
:10043000AA233430BC2347222508031D252A24087B
:10044000803C031C252A1C2122154B223B23003013
:10045000AF232B30211E2D30BC234D30AF23221C67
:10046000332A4D30342A4130BC232A30BC23BC23EC
:10047000ED23221DC3282211B1231D302218422A48
:100480003223C3280130AF234D30BC23C32846306C
:1004900032234A30322BA210213084008403040816
:1004A000183C03190800A21808005A22A2180800D4
:1004B00071224E2A0008F0399000100E003C0319FA
:1004C0006B2A100E0D3C03196B2A100E0A3C0319FF
:1004D0006B2AA2140800000EF0390A388000800E42
:1004E0000800A2180800800E5A22800E08008B0116
:1004F000ED22A21D842AAA231D3022183A3032236D
:10050000EC23AA232E303223A21121100618892AA7
:10051000AD2A83160113831206189D2ACC20B60A31
:10052000031D9B2AB70A031D9B2AB80A381D9B2A64
:10053000A2152621772A061C8E2ACC20B60A031D76
:10054000AA2AB70A031DAA2AB80A381DAA2AA21580
:100550002621772A06189D2AD12A8316011783128D
:100560000618C12ACC20B60A031DBF2AB70A031DEC
:10057000BF2AB80A381DBF2AA2152621772A0618D5
:10058000B22ACC20B60A031DCE2AB70A031DCE2AF2
:10059000B80A381DCE2AA2152621772A061CC12AA0
:1005A000D12A81018B010B168B16A11121108B17FB
:1005B0008101CC204E30AF23A11EE42A2030BC2381
:1005C000FF30BC23A112E92AFF30BC232030BC231A
:1005D000A116ED23A11DD92A08001930840080013D
:1005E000840A0408213C031DEF2AA501A401A301EC
:1005F000B601B701B801080001308F000030920049
:100600000F08031908000310120C193E8400DF3E86
:100610000319080012180F2B1223920A002B2E2305
:10062000920A002B0F3000058F070F08F63E0319C2
:10063000212B0318262BF03080050F0880048F0132
:100640000800F03080058F018F0A08008F00F0301D
:1006500080050F0880048F018F0A0800800E122386
:10066000800E080090003720003E03190800BC23CC
:10067000900A1008332BAD230830910020308400FD
:10068000000E2520BC2300082520BC2384039103F1
:1006900003190800402B043090000D305A2B0C3009
:1006A00090000A305A2B0C3090000E305A2B0F302D
:1006B00090000F3097002030840010080319712B30
:1006C000800E0008F039800090030319782B840312
:1006D000000E0F39840A8004840390030319712BE0
:1006E000602B00080F398000170EF03980040800D5
:1006F0000008F039800017080F3980040800EE2345
:100700003030F039980016080F39180486000615A5
:1007100000000611080010307F2301307F230130D4
:10072000EE232030F039980016080F39180486009F
:100730000615000006110130EE232830BF230C30CF
:10074000BF23A5230630BF2308000130BF2BAD23F4
:10075000B323AD2BB123B323B12B0230BF2B803891
:10076000BF2BC030BF2B103090002030BC23900333
:100770009008031DB52B08009615C5230800961197
:10078000C5230430EE231708080097000130E32347
:1007900016111708F039980016080F39180486004A
:1007A000061500000611970E1708F0399800160874
:1007B0000F3918048600061500000611961516114B
:1007C000970E17080800413093009303031DE52B93
:1007D0000800ED23ED23ED23ED23C8309300930AA9
:1007E000930BF32B08009401940BF42B4C309400E2
:0607F000940BF82BF02B26
:02400E00F13F80
:1042000043006F0070007900720069006700680069
:104210007400200031003900390039002E002000E0
:10422000440065007300690067006E00650064006B
:10423000200061006E0064002000570072006900D9
:104240007400740065006E00200062007900200098
:10425000460072002E00200054006F006D00200008
:0E4260004D00630047006100680065006500C6
:00000001FF
